:020000040800F2
:1000000038300020CD010008512900082B240008B9
:10001000212900088104000889350008000000003B
:10002000000000000000000000000000852D000816
:100030007D0500080000000055290008592E000821
:10004000E7010008E7010008E7010008E7010008F0
:10005000E7010008E7010008E7010008E7010008E0
:10006000E7010008E7010008E7010008E7010008D0
:10007000E7010008E7010008E7010008E7010008C0
:1000800041050008E7010008E7010008E701000852
:10009000E7010008E7010008E7010008E7010008A0
:1000A000E7010008E7010008E7010008E701000890
:1000B000652E0008E7010008E7010008E7010008D5
:1000C000E7010008E7010008E7010008E701000870
:1000D000E70100086935000879350008E7010008E4
:1000E000E7010008E7010008E7010008E701000850
:1000F000E7010008E7010008E7010008E701000840
:10010000E7010008E7010008E7010008E70100082F
:10011000E7010008E7010008E7010008E70100081F
:10012000E7010008E7010008E7010008E70100080F
:1001300000F002F800F03AF80AA090E8000C8244BF
:100140008344AAF10107DA4501D100F02FF8AFF29C
:10015000090EBAE80F0013F0010F18BFFB1A43F0A5
:1001600001031847943E0000B43E0000103A24BF3B
:1001700078C878C1FAD8520724BF30C830C144BF0C
:1001800004680C607047000000230024002500264E
:10019000103A28BF78C1FBD8520728BF30C148BFEA
:1001A0000B6070471FB51FBD10B510BD00F0E8F81B
:1001B0001146FFF7F7FF03F0B3FC00F006F903B4B4
:1001C000FFF7F2FF03BC03F089FA000009488047FB
:1001D00009480047FEE7FEE7FEE7FEE7FEE7FEE729
:1001E000FEE7FEE7FEE7FEE704480549054A064B41
:1001F00070470000612E000831010008382A0020F5
:1002000038300020382C0020382C00207047B2F104
:1002100020030AD5C2F1200320FA02F001FA03F309
:1002200021FA02F140EA0300704721FA03F04FF08F
:1002300000017047032A40F2308010F0030C00F0F8
:10024000158011F8013BBCF1020F624498BF11F810
:1002500001CB00F8013B38BF11F8013BA2F10402C9
:1002600098BF00F801CB38BF00F8013B11F0030341
:1002700000F02580083AC0F0088051F8043B083AA5
:1002800051F804CBA0E80810F5E7121D5CBF51F847
:10029000043B40F8043BAFF30080D20724BF11F8C1
:1002A000013B11F801CB48BF11F8012B24BF00F826
:1002B000013B00F801CB48BF00F8012B704710B597
:1002C000203AC0F00B80B1E81850203AA0E818504E
:1002D000B1E81850A0E81850BFF4F5AF5FEA027C0F
:1002E00024BFB1E81850A0E8185044BF18C918C07E
:1002F000BDE810405FEA827C24BF51F8043B40F81F
:10030000043B08BF7047D20728BF31F8023B48BF03
:1003100011F8012B28BF20F8023B48BF00F8012B41
:1003200070474FF0000200B51346944696462039B8
:1003300022BFA0E80C50A0E80C50B1F12001BFF49E
:10034000F7AF090728BFA0E80C5048BF0CC05DF804
:1003500004EB890028BF40F8042B08BF704748BF52
:1003600020F8022B11F0804F18BF00F8012B7047C6
:10037000704770477047704700487047D429002085
:100380007546FFF7F9FFAE4605006946534620F073
:100390000700854618B020B5FFF726FFBDE82040CE
:1003A0004FF000064FF000074FF000084FF0000B31
:1003B00021F00701AC46ACE8C009ACE8C009ACE8E4
:1003C000C009ACE8C0098D46704710B50446AFF3CC
:1003D00000802046BDE81040FFF7F1BE00200A492A
:1003E00000BF03E00A5C094B1A54401CB0F5486F8B
:1003F000F8D3D1F8802C054BC3F8802CD1F8842C8D
:10040000C3F8842C7047000000F00308CC100020D3
:1004100010B540F244620249024800F0CBF910BD29
:10042000CC10002000F0030810B50B480068401CF9
:10043000094908600846006844F62061884209D3EB
:1004400008460549086000BF01221146034801F033
:1004500009F800BF10BD000028000020000C01407A
:1004600010B500BF00220121034800F0FBFF00BFD0
:1004700000200249086010BD000C01402800002047
:1004800000BFFEE7F0B502460C46FF21FF2509E05C
:1004900012F8016B86EA0103084EF65C86EA050154
:1004A000074EF55C261EA4F10107BCB2F0D1084648
:1004B0004FF6FF7606EA00202843F0BDF83D00081D
:1004C000F83E0008F0B505460C46A01E2E5C4FF61F
:1004D000FF7000EA0626601E285C0643A01E81B25B
:1004E0002846FFF7CFFF0746BE4201D10120F0BDED
:1004F0000020FCE770B500BFD52003F069F800BF0D
:100500000021084602F08CFC002416E000250DE0D6
:10051000002003F093F8002003F090F8002003F08F
:100520008DF8002003F08AF8681C85B2142DEFDBEB
:10053000002003F083F8601C84B2A02CE6DB70BDC1
:1005400010B5024800F0AAFA10BD000044100020C7
:1005500030B590F840500124AC40C56B6C60046825
:1005600063604468102C04D10468A2600468E160F0
:1005700003E00468A1600468E26030BD70470000D9
:100580002DE9F84F81460F46904630A00068009054
:1005900000BFD52003F01CF800BFB9F1A00F01D8AF
:1005A000A02F01D9BDE8F88FC9F1A00040080321B0
:1005B000B0FBF1F000F0FF0AC7F1A00007EB50001C
:1005C00000F0FF0B4FEAD90600243BE0ABEB040040
:1005D000C1B2504602F024FC00252CE004FB065179
:1005E00018F80110C943C1F381111DF8010003F08F
:1005F00025F804FB065118F80110C943C1F3011195
:100600001DF8010003F01AF804FB065118F8011058
:10061000C943C1F381011DF8010003F00FF804FB89
:10062000065118F80120032191431DF8010003F041
:1006300005F8681CC5B2B542D0D3002002F0FEFF19
:10064000601CC4B2BC42C1D300BFABE7000FF0FFD7
:100650000021074AD1610749096941F00401054AAF
:1006600011611146096941F04001116170470000B4
:1006700060010020002002400021074AD1610749A3
:10068000096941F00201054A116111464861096991
:1006900041F04001116170476001002000200240DC
:1006A0000022054BDA61054A126942F00102034B50
:1006B0001A610180704700006001002000200240A4
:1006C00000201E49C96801F0100139B11C49C969EF
:1006D00041F002011A4AD16140F010001749C9687F
:1006E00001F0040139B11649C96941F00101144A08
:1006F000D16140F004001149C96901F0010169B1FB
:100700000F49C96941F004010D4AD16100BF0B498D
:10071000C96921F00101094AD16100BF00BF40F25F
:100720000111884206D10549C96921F00101034A36
:10073000D16101E00149C86000BF7047002002405C
:100740006001002070B5044600F092FE054609E005
:10075000601C38B124B100F08BFE401BA04201D9CF
:10076000032070BD1248C06800F001000028EFD1DE
:100770000F48C06800F0200020B100BF20200C49C5
:10078000C86000BF0A48C06800F0100048B90848B7
:10079000C06900F0010020B90548C06800F00400FD
:1007A00018B1FFF78DFF0120DBE70020D9E700003B
:1007B000002002402DE9F74F88B005469046A5F18C
:1007C0000060079007984FEAD02A4FF0006000EBD6
:1007D000CA26A81B06904FEA480705950698384494
:1007E0004FEAD02B4FF000090020009006983844C3
:1007F000C0F30A0008B10BF1010BB5F1006F03D390
:10080000E8192549884203D301200BB0BDE8F08FD9
:10081000B6F1006F02D32048864201D30120F4E7ED
:1008200000F056FC0598C11906F5006081422ED3F0
:10083000002414E0002001900396012004906946F2
:1008400001A800F08BFB8146B9F1000F03D000F046
:10085000DDFB4846D9E706F50066601C84B25C45BE
:10086000E8D3002410E0099830F814C005EB4401E7
:1008700062460023012000F0D3FB8146B9F1000F4E
:1008800000D003E0601C84B24445ECDB00BF00F004
:10089000BDFB4846B9E700000000040801460022FD
:1008A00091F82100022808D00420886300BF0020AE
:1008B00081F8200000BF012070470868006820F020
:1008C0000E000B6818600868006820F001000B68D3
:1008D000186091F8403001209840CB6B586001209F
:1008E00081F8210000BF002081F8200000BF1046E1
:1008F000E2E7000070B50446002594F821000228C4
:1009000003D00420A0630125C1E02068006820F026
:100910000E00216808602068006820F0010021684E
:1009200008605C492068884252D95A497839206861
:10093000884201D1012047E0564964392068884245
:1009400001D1102040E0534950392068884201D13C
:10095000801539E04F493C392068884201D1801424
:1009600032E04C4928392068884202D14FF4803067
:100970002AE0484914392068884202D14FF4801097
:1009800022E044492068884201D140041CE04249E9
:100990002068884201D1012016E03F4914312068C7
:1009A000884201D110200FE03B492831206888425D
:1009B00001D1801508E038493C312068884201D1D6
:1009C000801401E04FF480303349091F086051E082
:1009D000304978392068884201D1012047E02D490B
:1009E00064392068884201D1102040E029495039FB
:1009F0002068884201D1801539E026493C392068B9
:100A0000884201D1801432E0224928392068884286
:100A100002D14FF480302AE01E4914392068884200
:100A200002D14FF4801022E01A492068884201D197
:100A300040041CE018492068884201D1012016E0DA
:100A4000154914312068884201D110200FE0124965
:100A500028312068884201D1801508E00E493C31D8
:100A60002068884201D1801401E04FF480300949A8
:100A700080394860012084F8210000BF002084F8FC
:100A8000200000BF606B10B12046616B884728468C
:100A900070BD0000800002400804024070B50446AA
:100AA000E06B05682068066894F8401004208840D0
:100AB0002840002875D006F004000028FAD02068ED
:100AC000006800F0200028B92068006820F00400C9
:100AD00021680860D5492068884254D9D3497839BB
:100AE0002068884201D1042049E0D0496439206857
:100AF000884201D1402042E0CC49503920688842E8
:100B000001D100153BE0C9493C392068884202D137
:100B10004FF4804033E0C54928392068884202D12B
:100B20004FF480202BE0C14914392068884202D15B
:100B30004FF4800023E0BD492068884201D1C00401
:100B40001DE0BB492068884201D1042017E0B84964
:100B500014312068884201D1402010E0B449283186
:100B60002068884201D1001509E0B1493C31206874
:100B7000884202D14FF4804001E04FF48020AC491C
:100B8000091F086054E0A94978392068884201D1DA
:100B900004204AE0A54964392068884202D14020F7
:100BA00043E04CE0A14950392068884201D100154A
:100BB0003BE09E493C392068884202D14FF4804096
:100BC00033E09A4928392068884202D14FF48020C6
:100BD0002BE0964914392068884202D14FF48000F6
:100BE00023E092492068884201D1C0041DE0904969
:100BF0002068884201D1042017E08D491431206813
:100C0000884201D1402010E089492831206888427B
:100C100001D1001509E086493C312068884202D1A3
:100C20004FF4804001E04FF48020804980394860D3
:100C3000E06A002802D02046E16A8847F4E094F890
:100C40004010022088402840002871D006F00200A1
:100C50000028FAD02068006800F0200040B9206821
:100C6000006820F00A0021680860012084F8210053
:100C70006E492068884254D96C4978392068884286
:100C800001D1022049E0694964392068884201D1D4
:100C9000202042E0654950392068884201D1401542
:100CA0003BE062493C392068884202D14FF4005051
:100CB00033E05E4928392068884202D14FF4003081
:100CC0002BE05A4914392068884202D14FF40010B1
:100CD00023E056492068884201D180041DE0544930
:100CE0002068884201D1022017E051491431206860
:100CF000884201D1202010E04D49283120688842E7
:100D000001D1401509E04A493C312068884202D1AE
:100D10004FF4005001E04FF400304549091F0860CE
:100D200054E0424978392068884202D102204AE0E2
:100D300057E03E4964392068884201D1202042E0D2
:100D40003A4950392068884201D140153BE0374983
:100D50003C392068884202D14FF4005033E03349D7
:100D600028392068884202D14FF400302BE02F4907
:100D700014392068884202D14FF4001023E02B4937
:100D80002068884201D180041DE0294920688842FA
:100D900001D1022017E0264914312068884201D190
:100DA000202010E0224928312068884201D14015D6
:100DB00009E01F493C312068884202D14FF40050BD
:100DC00001E04FF4003019498039486000BF00202D
:100DD00084F8200000BFA06A30B32046A16A88478B
:100DE00022E094F84010082088402840E0B106F046
:100DF0000800C8B12068006820F00E002168086073
:100E000094F8401001208840E16B48600120A06305
:100E100084F8210000BF002084F8200000BF206B70
:100E200010B12046216B884770BD00008000024051
:100E3000080402400146002209B9012070471E4BF8
:100E4000086898420BD21D4B0868C01A1423B0FBE7
:100E5000F3F08000086419480838C8630AE0164BAC
:100E60000868C01A1423B0FBF3F08000086412482D
:100E70000838C863022081F821000868026843F638
:100E8000F0708243D1E901031843CB6818430B6922
:100E900018434B6918438B691843CB6918430243C5
:100EA0000868026000208863012081F8210000208A
:100EB00081F8200000BFC1E708040240080002409A
:100EC0002DE9F04104460D4616461F464FF0000836
:100ED00000BF94F82000012802D10220BDE8F08173
:100EE000012084F8200000BF94F8210001282CD1B3
:100EF000022084F821000020A0632068006820F010
:100F00000100216808603B46324629462046FFF72B
:100F10001FFBE06A30B12068006840F00E002168D5
:100F200008600BE02068006820F004002168086079
:100F30002068006840F00A002168086020680068A6
:100F400040F001002168086006E000BF002084F83E
:100F5000200000BF4FF002084046BFE72DE9F041F6
:100F600004460E460127002500BF2648007E0128C2
:100F700002D10220BDE8F08101202249087600BF9D
:100F80002068022813D14CF25030FFF7DBFB90BBF6
:100F90000120FFF75DFB4CF25030FFF7D3FB074613
:100FA0001948006920F004001749086123E04CF259
:100FB0005030FFF7C7FBF0B94FF0FF303060A56845
:100FC00012E02846FFF758FB4CF25030FFF7BAFB0F
:100FD00007460D48006920F002000B4908610FB177
:100FE000356007E005F50065D4E9021001EBC0208B
:100FF000A842E6D800BF00BF00200249087600BF23
:101000003846B7E76001002000200240034800692D
:1010100040F0800001490861002070470020024034
:101020002DE9FE4F05468B461746984601260024BB
:101030000020029000BF2448007E012802D1022037
:10104000BDE8FE8F01202049087600BF4CF25030E9
:10105000FFF778FB064686BB012D02D101200290E6
:1010600006E0022D02D10220029001E0042002904D
:1010700000241EE02201B946C24648465146FFF709
:10108000C6F880B20190022000FB04B000900199E4
:10109000FFF706FB4CF25030FFF754FB06460B48B7
:1010A000006920F001000949086106B104E0601CF4
:1010B000C4B202988442DDDB00BF00BF00200249B9
:1010C000087600BF3046BBE76001002000200240E8
:1010D00000200849096901F0800151B10649054A1B
:1010E0005160064951601146096901F0800101B162
:1010F000012070470020024023016745AB89EFCDF6
:101100002DE9F847024600239C467BE14FF0010899
:1011100008FA03F4D1F8008008EA0400A0427DD167
:10112000DFF8F4A2D1F80480A8EB0A09D0453AD040
:1011300014DCB8F1030F50D009DCB8F1000F31D046
:10114000B8F1010F1CD0B8F1020F49D120E0B8F17D
:10115000110F18D0B8F1120F42D11EE0B9F5881F57
:1011600025D006DCB9F5803F20D0B9F5801F37D1F6
:101170001AE0B9F5001F18D0B9F5041F30D117E0F7
:10118000D1F80CC02DE0D1F80C8008F1040C28E057
:10119000D1F80C8008F1080C23E0D1F80C8008F19C
:1011A0000C0C1EE000BF00BF00BF00BF00BF00BFAF
:1011B000D1F80880B8F1000F02D14FF0040C0BE019
:1011C000D1F80880B8F1010F03D14FF0080C146179
:1011D00002E04FF0080C546103E04FF0000C00E017
:1011E00000BF00BFFF2801D8904601E002F10408CB
:1011F0004646FF2802D84FEA830803E0A3F1080817
:101200004FEA88084746D6F800804FF00F0909FAE0
:1012100007F928EA09080CFA07F900E07AE048EA39
:101220000908C6F80080D1F8048008F08058B8F1A9
:10123000805F6FD100BFDFF8E481D8F8188048F0F4
:101240000108DFF8D891C9F81880C846D8F8188086
:1012500008F00108CDF8008000BF00BF4FEAB938A0
:101260004FEA930958F829504FEA83784FEA1879E2
:101270004FF00F0808FA09F825EA0805DFF8A08101
:10128000424502D14FF0000824E0DFF89881424542
:1012900002D14FF001081DE0DFF88C81424502D1F8
:1012A0004FF0020816E0DFF88481424502D14FF08A
:1012B00003080FE0DFF87881424502D14FF00408BF
:1012C00008E0DFF87081424502D14FF0050801E0E7
:1012D0004FF006084FEA83794FEA197908FA09F8BE
:1012E00048EA0505DFF850814FEA930948F829508C
:1012F000D1F8048008F48018B8F5801F0BD1DFF80E
:101300003C81D8F8008048EA0008DFF83091C9F83D
:1013100000800AE075E0DFF82481D8F8008028EA30
:101320000008DFF81891C9F80080D1F8048008F4AB
:101330000018B8F5001F0ED1DFF8008108F104088D
:10134000D8F8008048EA0008DFF8F09009F10409B5
:10135000C9F800800DE0DFF8E48008F10408D8F84F
:10136000008028EA0008DFF8D49009F10409C9F8E0
:101370000080D1F8048008F40038B8F5003F0ED1A1
:10138000DFF8B880A8F10408D8F8008048EA00081F
:10139000DFF8A890A9F10409C9F800800DE0DFF892
:1013A0009C80A8F10408D8F8008028EA0008DFF83B
:1013B0008C90A9F10409C9F80080D1F8048008F4E0
:1013C0008038B8F5803F0ED1DFF87080A8F10808AA
:1013D000D8F8008048EA0008DFF86090A9F1080911
:1013E000C9F800800DE0DFF85480A8F10808D8F8AB
:1013F000008028EA0008DFF84490A9F10809C9F83C
:1014000000805B1CD1F8008028FA03F8B8F1000FC7
:101410007FF47CAEBDE8F887000011100010024098
:1014200000080140000C0140001001400014014080
:1014300000180140001C0140080001400804014060
:10144000024693680B400BB1012000E0002070477A
:1014500010B5C26821EA020302EA010443EA044328
:10146000036110BD0AB1016101E00B040361704723
:101470000148006870470000180000200348006819
:1014800003490978084401490860704718000020A2
:101490002000002010B50848006840F01000064900
:1014A0000860032000F080F80F2000F007F800F03B
:1014B0002BF8002010BD00000020024070B504464B
:1014C0000E4800784FF47A71B1FBF0F00C490968CE
:1014D000B1FBF0F5284600F0F3FB08B1012070BD28
:1014E000102C07D200222146501E00F01EF805489D
:1014F000046001E00120F2E70020F0E72000002076
:10150000080000201C000020704701460846002803
:1015100009DB00F01F0301229A4043099B0003F1FD
:10152000E023C3F8002100BF70472DE9F05F80463B
:101530000D461646002702F0B5F8074639462A46FA
:10154000334601F00700C0F1070ABAF1040F02D9CF
:101550004FF0040A01E0C0F1070AD14600F1040A85
:10156000BAF1070F02D24FF0000A01E0A0F1030A1E
:10157000D4464FF0010A0AFA09FAAAF1010A0AEA66
:10158000020A0AFA0CFA4FF0010B0BFA0CFBABF152
:10159000010B0BEA030B4AEA0B042146404602F01A
:1015A00089F8BDE8F09F000000BF00F00702064B7D
:1015B00019684FF6FF031940044B0B4343EA02211D
:1015C000014B196000BF70470CED00E00000FA0508
:1015D00000BF00BF00BF00BF00BFBFF34F8F00BF01
:1015E00000BF00BF0948006800F4E06008490843F4
:1015F000001D0649086000BF00BF00BFBFF34F8F4A
:1016000000BF00BF00BF00BF00BFFDE70CED00E062
:101610000000FA0570B504460D460CB9012070BDF6
:101620005A48006800F00700A8420ED257480068E8
:1016300020F007002843554908600846006800F07C
:101640000700A84201D00120E9E7207800F002005D
:1016500002281DD1207800F00400042805D14C4850
:10166000406840F4E0604A494860207800F0080093
:10167000082805D14648406840F460504449486015
:101680004348406820F0F000A168084340494860A2
:10169000207800F0010078B36068012806D13C484A
:1016A000006800F4003090B90120B8E760680228B3
:1016B00006D13748006800F0007040B90120AEE75D
:1016C0003348006800F0020008B90120A7E730485D
:1016D000406820F00300616808432D494860FFF727
:1016E000C7FE064609E0FFF7C3FE801B41F28831C2
:1016F000884202D9032092E707E02548406800F0BD
:101700000C006168B0EB810FEDD12048006800F05B
:101710000700A8420ED91D48006820F007002843A2
:101720001A4908600846006800F00700A84201D086
:10173000012074E7207800F00400042807D1144841
:10174000406820F4E060E16808431149486020786F
:1017500000F00800082808D10D48406820F46050C7
:10176000216940EAC1000A49486000F03FF8084991
:101770004968C1F30311074A515CC8400649086033
:1017800006480068FFF79AFE002048E70020024064
:1017900000100240223C0008080000201C0000202D
:1017A00001480068704700000800002000B5FFF7FE
:1017B000F7FF04494968C1F30221034A515CC8405C
:1017C00000BD000000100240323C000800B5FFF7E9
:1017D000E7FF04494968C1F3C221034A515CC8408C
:1017E00000BD000000100240323C000870B500212E
:1017F0000022002400230020134D696801F00C052D
:10180000F5B1042D02D0082D19D101E00F4819E0DF
:101810000F4DC1F38346AB5D01F4803555B10A4DE0
:101820006D68C5F340450B4E725D084D5D43B5FBD9
:10183000F2F402E0084D03FB05F4204602E000BF8D
:10184000024800BF00BF70BD0010024000127A00C5
:101850003A3C00084A3C000800093D00F8B504463F
:101860000CB90120F8BD207800F00100002878D0E4
:10187000F848406800F00C0004280CD0F548406897
:1018800000F00C00082811D1F248406800F48030C4
:10189000B0F5803F0AD1EF48006800F4003000281E
:1018A0005FD0606800285CD10120DBE700BF606882
:1018B000B0F5803F06D1E748006840F48030E54944
:1018C000086028E0606858B9E248006820F4803079
:1018D000E04908600846006820F4802008601AE0AB
:1018E0006068B0F5A02F0BD1DA48006840F4802082
:1018F000D84908600846006840F4803008600AE073
:10190000D448006820F48030D24908600846006856
:1019100020F48020086000BF606888B1FFF7A8FD50
:10192000054606E0FFF7A4FD401B642801D903200B
:1019300098E7C848006800F400300028F2D010E0B2
:10194000FFF796FD054606E0FFF792FD401B642871
:1019500001D9032086E7BF48006800F40030002862
:10196000F2D1207800F00200022857D1B94840682F
:1019700000F00C0050B1B748406800F00C00082897
:1019800018D1B448406800F4803098B9B148006874
:1019900000F0020020B12069012801D0012061E798
:1019A000AC48006820F0F800616940EAC100A9492C
:1019B000086033E02069E8B10120A7490860FFF71B
:1019C00057FD054606E0FFF753FD401B022801D9ED
:1019D000032047E79F48006800F002000028F2D08B
:1019E0009C48006820F0F800616940EAC10099490C
:1019F000086013E0002098490860FFF739FD0546AC
:101A000006E0FFF735FD401B022801D9032029E736
:101A10009048006800F002000028F2D1207800F021
:101A2000080008282DD1A069B8B101208B490860B1
:101A3000FFF71EFD054606E0FFF71AFD401B0228D2
:101A400001D903200EE78348406A00F00200002815
:101A5000F2D0012000F09CFF13E000207F490860D5
:101A6000FFF706FD054606E0FFF702FD401B0228D2
:101A700001D90320F6E67748406A00F0020000280A
:101A8000F2D1207800F00400042873D100277148B7
:101A9000C06900F0805070B900BF6E48C06940F066
:101AA00080506C49C8610846C06900F080500090C1
:101AB00000BF00BF01276A48006800F48070B0B919
:101AC0006748006840F4807065490860FFF7D0FC03
:101AD000054606E0FFF7CCFC401B642801D9032033
:101AE000C0E65F48006800F480700028F2D000BFB4
:101AF000E068012806D15748006A40F001005549C6
:101B0000086227E0E06858B95248006A20F00100F6
:101B1000504908620846006A20F00400086219E093
:101B2000E06805280BD14B48006A40F004004949A1
:101B300008620846006A40F0010008620AE0454871
:101B4000006A20F00100434908620846006A20F05C
:101B50000400086200BFE068A0B1FFF789FC0546F9
:101B600009E0FFF785FC401B41F28831884202D929
:101B7000032077E622E03748006A00F002000028E0
:101B8000EFD012E0FFF774FC054608E0FFF770FCA9
:101B9000401B41F28831884201D9032062E62D487A
:101BA000006A00F002000028F0D1012F05D1294879
:101BB000C06920F080502749C86100BFE069C8B300
:101BC0002448406800F00C00082860D0E069022832
:101BD00048D1002020490866FFF74AFC054606E088
:101BE000FFF746FC401B022801D903203AE61948BA
:101BF000006800F000700028F2D1206AB0F5803F44
:101C000007D11448406820F40030A1680843114906
:101C10004860D4E9080108430E49496821F4741169
:101C200008430C49486001200B490866FFF720FC77
:101C3000054607E03DE0FFF71BFC401B022801D9E9
:101C400003200FE60348006800F000700028F2D07F
:101C50002FE0000000100240000042428004424297
:101C600000700040002014490866FFF701FC05469B
:101C700006E0FFF7FDFB401B022801D90320F1E538
:101C80000E48006800F000700028F2D111E0E06911
:101C9000012800D1E6E50948466806F48031206A4B
:101CA000814204D106F47011606A814201D00120A2
:101CB000D8E50020D6E500000000424200100240B6
:101CC00070B504462546681EB0F1807F01D301201F
:101CD0000FE0681E4FF0E02148610F214FF0FF3008
:101CE00001F0E8FC00204FF0E02188610720086146
:101CF000002070BD10B504460CB9012010BD94F849
:101D00003D0028B9002084F83C00204600F025F86A
:101D1000022084F83D00211D206801F0D5F8012043
:101D200084F8460000BF84F83E0001213F200155A1
:101D3000402001554120015500BF00BF012084F81B
:101D4000420043200155442001554520015500BF64
:101D5000012084F83D000020D0E77047014691F84B
:101D60003D00012801D001207047022081F83D008C
:101D70000868C06840F001000B68D860164B08681E
:101D8000984213D0154B086898420FD00868B0F1FC
:101D9000804F0BD0124B0868984207D0114B08684F
:101DA000984203D0104B086898420CD108688068AC
:101DB00000F00702062A0CD00868006840F0010015
:101DC0000B68186005E00868006840F001000B68C7
:101DD00018600020C8E70000002C014000340140DA
:101DE0000004004000080040000C0040F8B5044624
:101DF0000D46164694F8420020282DD105B10EB9A3
:101E00000120F8BD0120206300206063324629468E
:101E1000204601F0A3FA0746206B012819D100BF24
:101E200000200090206800680090206840680090C2
:101E300000BF00BF00BF00BF21680C3151E8001F88
:101E400041F0100021680C3141E80002002AF3D172
:101E500000E001273846D4E70220D2E770B50446F7
:101E60000D4607492068884208D1012005490870BD
:101E700040F68842491C0448FFF7B8FF70BD0000D7
:101E80000044004068030020FC0F00207047000061
:101E90002DE9F84F0446206805682068C668206868
:101EA00047694FF00009CA4605F00F09B9F1000F64
:101EB0000AD105F0200038B106F0200020B12046FC
:101EC00001F04FF9BDE8F88FB9F1000F7BD007F0B2
:101ED000010018B906F49070002874D005F00100D4
:101EE00030B106F4807018B1606C40F0010060649D
:101EF00005F0040030B107F0010018B1606C40F04B
:101F00000200606405F0020030B107F0010018B172
:101F1000606C40F00400606405F0080048B106F011
:101F2000200010B907F0010018B1606C40F0080003
:101F30006064606C002845D005F0200028B106F0F0
:101F4000200010B1204601F00CF920684069C0F370
:101F5000801A606C00F0080010B9BAF1000F2CD0A4
:101F6000204601F0A5F82068406900F0400000B369
:101F700000BF00BF2168143151E8001F21F040006C
:101F80002168143141E80002002AF3D100BFE06B60
:101F900050B17748E16B4863E06BFEF7ABFC88B16A
:101FA000E06B416B88470DE02046FFF76FFF09E0CB
:101FB00009E02046FFF76AFF04E02046FFF766FFCE
:101FC000002060647EE7206B012877D105F01000C7
:101FD000002873D006F010000028FAD000BF0020BF
:101FE000009020680068009020684068009000BF62
:101FF00000BF2068406900F0400000285FD0E06B1F
:10200000006840681FFA80F8B8F1000F55D0A08D25
:10201000404552DDA4F82E80E06B8069202843D033
:1020200000BF00BF21680C3151E8001F21F480700F
:1020300021680C3141E80002002AF3D100BF00BF43
:1020400000BF2168143151E8001F21F00100216810
:10205000143141E80002002AF3D100BF00BF00BFE5
:102060002168143151E8001F21F04000216814312B
:1020700041E80002002AF3D100BF202084F842008A
:102080000020206300BF00BF21680C3151E8001F11
:1020900021F0100021680C3141E80002002AF3D140
:1020A00000BFE06BFEF7FAFB02206063A08DE28DBB
:1020B000801A81B22046FFF7D1FE03E742E0A08DEF
:1020C000E18D401A1FFA80F8E08DD0B3B8F1000F0F
:1020D00037D000BF00BF21680C3151E8001F21F448
:1020E000907021680C3141E80002002AF3D100BF52
:1020F00000BF00BF2168143151E8001F21F001002A
:102100002168143141E80002002AF3D100BF2020E9
:1021100084F842000020206300BF00BF21680C311A
:1021200051E8001F21F0100021680C3141E8000245
:10213000002AF3D100BF0220606341462046FFF72A
:102140008DFEBFE605F0800030B106F0800018B1CA
:10215000204601F087F9B5E605F0400030B106F001
:10216000400018B1204600F0D9FFABE600BFA9E659
:10217000752F000810B504460CB9012010BDA069E8
:1021800000B100E000BF94F8410028B9002084F8B5
:102190004000204600F02AF8242084F841002068FE
:1021A000C06820F400502168C860204601F058F84B
:1021B0002068006920F49040216808612068406927
:1021C00020F02A00216848612068C06840F400506F
:1021D0002168C86000206064202084F8410084F8F1
:1021E00042000020606300BFC8E7000010B586B061
:1021F00004462849206888424AD100BF00BF2648CB
:10220000806940F00400244988610846806900F034
:102210000400019000BF00BF00BF00BF00BF084620
:10222000806940F0040088610846806900F004007D
:10223000019000BF00BF00BF00BF00BF084680691B
:1022400040F4804088610846806900F48040019035
:1022500000BF00BF00BF481502900220039001207C
:1022600004900320059002A90C48FEF749FF4FF4A3
:10227000806002900020039002A90848FEF740FF0A
:102280002520FFF742F9032211462520FFF74DF9DB
:1022900006B010BD003801400010024000080140A7
:1022A00070B504460D46164694F8420020280BD11E
:1022B00005B10EB9012070BD0020206332462946C9
:1022C000204601F0AFF8F6E70220F4E710B5044627
:1022D0002049206888423BD11F48008800F4004014
:1022E00088BB1D48008800F4804070B11B4800780E
:1022F0000A2803D000201849088024E016480088E6
:1023000040F40040144908801DE0144800780D286E
:1023100006D11148008840F480400F49088012E03F
:102320000E4800780C490988C1F30D010C4A50543D
:1023300009480088401C0849088008460088C728CA
:1023400001DD00200880012204490648FFF7A8FFAC
:1023500010BD0000003801401400002016000020CD
:10236000500000201801002070472DE9F84F044666
:102370000E46174699464FF0000A94F8410020286F
:1023800050D106B117B90120BDE8F88F0020606474
:10239000212084F84100FFF76BF88246A784E78488
:1023A000A068B0F5805F04D1206910B90025B0465F
:1023B00002E035464FF000081EE05346002280211F
:1023C0002046CDF8009001F07DF820B1202084F85F
:1023D00041000320D8E745B9B8F80000C0F3080071
:1023E0002168486008F1020803E028782168486005
:1023F0006D1CE08C401EE084E08C0028DDD153464B
:10240000002240212046CDF8009001F05BF820B179
:10241000202084F841000320B6E7202084F8410002
:102420000020B1E70220AFE7704700BFFEE70000E1
:1024300008B5434A811A904241D009DC4149014420
:1024400081B1B1F5806F1CD0B1F5006F74D127E078
:10245000B1F5806F42D0B1F5006F4ED0B1F5406F4D
:102460006AD159E000BF3849896941F00401364A10
:1024700091611146896901F00401009100BF00BF1C
:102480005BE000BF3049896941F008012E4A916143
:102490001146896901F00801009100BF00BF4CE0BE
:1024A00000BF2949896941F01001274A916111460D
:1024B000896901F01001009100BF00BF3DE000BF3D
:1024C0002149896941F020011F4A916111468969BA
:1024D00001F02001009100BF00BF2EE000BF1A49AB
:1024E000896941F04001184A91611146896901F0FA
:1024F0004001009100BF00BF1FE000BF1249896981
:1025000041F08001104A91611146896901F0800112
:10251000009100BF00BF10E000BF0B49896941F482
:102520008071094A91611146896901F480710091B5
:1025300000BF00BF01E0FFE700BF00BF08BD000013
:102540000014014000F8FEBF001002401FB500203B
:1025500001900120029003200390002418E004EB76
:102560004401204A02EB81014868FFF761FF04EB58
:1025700044001C4931F82000009004EB4401194A42
:1025800002EB810148686946FEF7BAFD601CC4B2DF
:10259000092CE4D3002421E004EB440101EBC40145
:1025A000114A02EB810023460022104901F0F2F9A2
:1025B00004EB440101EBC4010B4A02EB81000C4A1D
:1025C000032101F08DF804EB440101EBC401064A3C
:1025D00002EB810001F01AFA601CC4B2092CDBD3B3
:1025E0001FBD00008C3D0008DC010020E53900081B
:1025F000F536000810B50446FDF732FF01480470B7
:1026000010BD00000500002001490860704700006F
:102610002400002008B5434A811A904241D009DCC9
:102620004149014481B1B1F5806F1CD0B1F5006F13
:1026300074D127E0B1F5806F42D0B1F5006F4ED074
:10264000B1F5406F6AD159E000BF3849896941F05E
:102650000401364A91611146896901F00401009133
:1026600000BF00BF5BE000BF3049896941F008014D
:102670002E4A91611146896901F00801009100BF5D
:1026800000BF4CE000BF2949896941F01001274A89
:1026900091611146896901F01001009100BF00BFEE
:1026A0003DE000BF2149896941F020011F4A916145
:1026B0001146896901F02001009100BF00BF2EE0A2
:1026C00000BF1A49896941F04001184A91611146D9
:1026D000896901F04001009100BF00BF1FE000BF09
:1026E0001249896941F08001104A91611146896956
:1026F00001F08001009100BF00BF10E000BF0B4956
:10270000896941F48071094A91611146896901F42E
:102710008071009100BF00BF01E0FFE700BF00BF74
:1027200008BD00000014014000F8FEBF0010024088
:102730001FB5002447E0274901EB04110868FFF7A3
:1027400069FF244800EB041080880090012001906C
:10275000204800EB0410806803901E4800EB041032
:10276000C06802901B4901EB041108686946FEF736
:10277000C7FC184B03EB0413DA79164B03EB041375
:102780009988144B03EB04131868FEF76BFE11488D
:1027900000EB0410807950B90E4800EB0410C079AA
:1027A00008B9012000E000200B49085509E009485C
:1027B00000EB0410C079012800D100E00020064998
:1027C0000855601CC4B2142CB5DB0121002000F0B8
:1027D0006FF81FBD4C3C00088001002070B5044616
:1027E000142C00DB70BD0C4800EB0410807908B994
:1027F000012500E00025084A02EB04129188064AF0
:1028000002EB041210682A46FEF72CFE0020034952
:10281000085500BFE6E700004C3C0008800100209E
:1028200070B50446142C00DB70BD0C4800EB04109E
:10283000807908B9002500E00125084A02EB04125E
:102840009188064A02EB041210682A46FEF70AFE37
:1028500001200349085500BFE6E700004C3C000892
:10286000800100202DE9F0410446E0780006A178BF
:1028700040EA0140617840EA0120217840EA0106FF
:1028800000250121002000F013F801250CE00120B3
:10289000A840304008B1012000E000200746E8B21F
:1028A000394600F005F86D1C142DF0D3BDE8F08119
:1028B00070B505460C46012C03D12846FFF7B0FF42
:1028C00002E02846FFF78AFF70BD000010B50446FD
:1028D000142C00DB10BD0A4A02EB04129188084A4E
:1028E00002EB04121068FEF7B3FD0648005D0128F4
:1028F00001D0012000E000200249085500BFE9E7AF
:102900004C3C00088001002010B5044AD2F8841C19
:10291000D2F8800CFDF734FE10BD0000CC10002072
:1029200000BFFEE710B5FDF759FDFFF7EDFF4FF4CF
:10293000FA7001F099F84FF4FA7001F095F84FF43D
:10294000FA7001F091F84FF4FA7001F08DF810BDB3
:1029500000BFFEE77047000006480078401C0549AC
:1029600008700846007918B108464079401C487143
:10297000704700003400002000200449887108716D
:102980004871C87101204880704700003400002061
:1029900008B508490968C9084FF47A72B1FBF2F129
:1029A0004143009100BF00BF00994A1E00920029D8
:1029B000F9D108BD0800002000B585B000BF00BFF8
:1029C0005348806940F00400514988610846806995
:1029D00000F00400009000BF00BF00BF00BF00BFB8
:1029E0000846806940F0040088610846806900F06C
:1029F0000400009000BF00BF00BF00BF00BF08463A
:102A0000806940F0040088610846806900F0040095
:102A1000009000BF00BF00BF00BF00BF0846C069F4
:102A200040F40030C8610846C06900F400300090EE
:102A300000BF00BF00BF00200190029003900490EF
:102A400004200190022002900120039003200490B2
:102A500001A93048FEF754FB0820019000200290A5
:102A600001A92C48FEF74CFB0220019001200290A6
:102A700001A92848FEF744FB2748284908600020A0
:102A800048600021254881608021C16000210161EA
:102A9000416181614FF44051C161FEF7CBF900BF44
:102AA0001E481F49C86308461C49486200BF1020E1
:102AB000FEF72BFD002211461020FEF736FD1948C7
:102AC0001749086018484860002115488160C160B6
:102AD000016181610C2141610021C161FFF74AFB65
:102AE0002620FEF712FD002201212620FEF71DFD03
:102AF00000BF012202210748FEF7B4FC00BF40F6E8
:102B000088420A490648FFF771F905B000BD000088
:102B100000100240000801406C00024044100020F8
:102B2000FC0F00200044004060AE0A006903002052
:102B300070B504460D462E462CB15D480078A04283
:102B400001D05B4804705B480078002876D00020F4
:102B500058490870012640F688415648401CFDF748
:102B6000B1FC012854D10020534908604FF4486259
:102B70005049491C5148FDF75DFB514951480268D5
:102B80000A604068486008460079892834D10846C0
:102B90004079452830D14FF4486248494A48FDF70A
:102BA0008EFB474840784649097840EA012046496B
:102BB000C1F8800C4248C0784149897840EA012038
:102BC0004149C1F8840CFDF723FCFDF749FCFDF7F2
:102BD00091FCFFF799FE4FF4FA7000F045FF4FF4B7
:102BE000FA7000F041FF4FF4FA7000F03DFF4FF42F
:102BF000FA7000F039FF19E034492E48D0F8810C02
:102C000008600846FFF72EFE2C4800F0BDF80DE0E6
:102C100029480068401C28490860084600680328C5
:102C200004D3FFF7C9FE002023490860002028498B
:102C3000887108714871C871012048802448408813
:102C400010B923488079B0B11948007838B11848D4
:102C50000178002000F082F80020154908701C4817
:102C60000078372807DD12480178012000F076F857
:102C700000200F49087016484079282808DD0120F7
:102C800013498871002048710846C079401CC871FA
:102C90000F48C079052808DB002605200C49C871BB
:102CA000FFF78AFE01200A494880304670BD0000C7
:102CB0003C000020680300204C000020541D002030
:102CC00041000020E90F0020CC1000203D00002032
:102CD000340000202DE9FC4104460D46164600272D
:102CE00001208DF800008DF801408DF802508DF81C
:102CF000036004216846FDF7C5FB074638128DF8CE
:102D00000400F8B28DF805000621684600F008F8C6
:102D1000002002494880BDE8FC810000340000200A
:102D200070B504460D4600BF002202210948FEF797
:102D300099FB00BFAAB24FF47A7321460648FFF709
:102D400014FB00BF012202210248FEF78BFB00BFEB
:102D500070BD000000080140FC0F002070B5044663
:102D60000D462A4621460320FFF7B4FF0020044900
:102D700048800870012008710020487170BD000073
:102D80003400002070470000F8B5064600BFD5208B
:102D900000F01EFC00BF21A0006800900021084642
:102DA00000F03EF8002436E000252DE004EB84011D
:102DB00005EB8101715C6A4602EB9111087800F025
:102DC0003DFC04EB840105EB8101715CC1F3011151
:102DD0001DF8010000F032FC04EB840105EB8101D9
:102DE000715CC1F381011DF8010000F027FC04EBC8
:102DF000840105EB8101715C01F003011DF8010004
:102E000000F01CFC681C85B2142DCFDB002000F004
:102E100015FC601C84B2A02CC6DBF8BD000FF0FFCF
:102E200070B504460D4604F12500C4B204F00F004D
:102E300000F0CEFBC4F3021141F0100000F0C8FB1B
:102E400005F00F0141F0600000F0C2FB702141EA83
:102E5000151000F0BDFB70BD10B5FEF70FFB10BDE7
:102E60007047000010B514480068006900F00100C8
:102E7000D8B112480068401C104908600846006834
:102E8000C821B0FBF1F201FB120010B901200C497E
:102E9000087000F0D5FD00BF01210A48FEF7D8FAFE
:102EA00000BFFDF7C1FAFFF757FD6FF001000249BF
:102EB0000968086110BD0000940100200000002096
:102EC000040000200008014010B50268244B98421D
:102ED0000ED0244B98420BD0B0F1804F08D0224B3B
:102EE000984205D0214B984202D0214B984203D101
:102EF00022F070024B681A43194B98420ED0194BBE
:102F000098420BD0B0F1804F08D0174B984205D0B3
:102F1000164B984202D0164B984203D122F44072CD
:102F2000CB681A4322F080034C6943EA0402026032
:102F30008B68C3620B688362094B984202D0094BCD
:102F4000984201D10B69036301234361036903F0D4
:102F500001031BB1036923F00103036110BD0000ED
:102F6000002C0140003401400004004000080040F3
:102F7000000C004070B505466C6A0020E085E084D6
:102F80002046FEF783FF70BD70B506460025746AC3
:102F900020684069C0F3C01594F84100212805D18C
:102FA00025B10020E084204600F0C8F82068406980
:102FB000C0F3801594F84200222805D125B10020E5
:102FC000E085204600F074F8606C40F0100060640A
:102FD0002046FEF75BFF70BD70B505466C6A286839
:102FE000006800F02000002842D1E08500BF00BF4B
:102FF00021680C3151E8001F21F4807021680C31E8
:1030000041E80002002AF3D100BF00BF00BF2168E1
:10301000143151E8001F21F001002168143141E80A
:103020000002002AF3D100BF00BF00BF21681431A5
:1030300051E8001F21F040002168143141E80002EE
:10304000002AF3D100BF202084F84200206B012821
:103050000ED100BF00BF21680C3151E8001F21F0E4
:10306000100021680C3141E80002002AF3D100BFB2
:1030700000206063206B012804D1A18D2046FEF75B
:10308000EDFE02E02046FFF721F970BD70B5054660
:103090006C6A01206063206B012805D1A08D410876
:1030A0002046FEF7DBFE02E02046FFF75DF970BD2B
:1030B00000BF00BF02680C3252E8002F22F490716A
:1030C00002680C3242E80013002BF3D100BF00BFAE
:1030D00000BF0268143252E8002F22F0010102689A
:1030E000143242E80013002BF3D100BF016B012919
:1030F0000ED100BF00BF02680C3252E8002F22F050
:10310000100102680C3242E80013002BF3D100BF1B
:10311000202180F8421000210163704710B5044659
:103120002068C06820F040002168C860202084F832
:1031300041002046FFF778F9002010BD00BF00BF16
:1031400002680C3252E8002F22F0C00102680C32F3
:1031500042E80013002BF3D100BF202180F841107A
:103160007047F8B5044694F84200222875D1A0684B
:10317000B0F5805F0CD1206950B90025A66A20689F
:103180004068C0F308003080A06A801CA06215E08F
:10319000A56A0026A068B0F5805F03D0A06828B9B2
:1031A000206918B920684068287004E020684068E9
:1031B00000F07F002870A06A401CA062E08D401ED5
:1031C00080B2E085002846D12068C06820F0200049
:1031D0002168C8602068C06820F480702168C860D9
:1031E0002068406920F0010021684861202084F8AF
:1031F000420000206063206B012826D1002020635C
:1032000000BF00BF21680C3151E8001F21F0100001
:1032100021680C3141E80002002AF3D100BF206888
:10322000006800F0100010280AD100BF00200090B4
:1032300020680068009020684068009000BF00BFD0
:10324000A18D2046FEF70AFE02E02046FFF73EF879
:103250000020F8BD01E00020FBE70220F9E70000B4
:1032600070B504462168096921F44051E2681143B0
:10327000226811612269A1681143626941EA02056D
:103280002168C96841F20C62914329432268D160E8
:103290002168496921F44071A26911432268516192
:1032A0002D4A2168914202D1FEF790FA01E0FEF723
:1032B0007DFA00EBC00101EB001162689200B1FBE6
:1032C000F2F100EBC00202EB001263689B00B2FB5C
:1032D000F3F26423B2FBF3F202EBC20303EB02123C
:1032E000A1EB8201322202EB01116422B1FBF2F167
:1032F00001F0F00100EBC00202EB001263689B00DA
:10330000B2FBF3F26423B2FBF3F201EB021200EB27
:10331000C00101EB001163689B00B1FBF3F100EB0E
:10332000C00303EB00136668B600B3FBF6F3642634
:10333000B3FBF6F303EBC30606EB0313A1EB830128
:10334000322303EB01116423B1FBF3F101F00F0110
:1033500011442268916070BD0038014077B581B09A
:10336000044615460298A062A585002060642220CC
:1033700084F842002848E16B88622848E16BC86203
:103380002748E16B08630020E16B486302AE3268B6
:103390002368191D2B46E06BFDF792FD00BF00204E
:1033A000009020680068009020684068009000BF8E
:1033B00000BF206970B100BF00BF21680C3151E827
:1033C000001F41F4807021680C3141E80002002A9E
:1033D000F3D100BF00BF00BF2168143151E8001FC6
:1033E00041F001002168143141E80002002AF3D1C4
:1033F00000BF00BF00BF2168143151E8001F41F039
:1034000040002168143141E80002002AF3D100BFD6
:10341000002004B070BD0000D92F00088D300008D6
:10342000892F000810B5034699629A85DA85002035
:103430005864222083F84200186928B11868C068CF
:1034400040F480701C68E0601868406940F001003A
:103450001C6860611868C06840F020001C68E0606B
:10346000002010BD014691F84100212828D188682C
:10347000B0F5805F0BD1086948B90A6A1088C0F3BB
:1034800008000B685860086A801C086205E00B6A37
:10349000581C086218780B685860C88C401E80B2AF
:1034A000C88458B90868C06820F080000B68D860EC
:1034B0000868C06840F040000B68D8600020704782
:1034C0000220FCE72DE9F84304460D4617469846CE
:1034D000089E31E0701C70B3FDF7CAFFA0EB080036
:1034E000B04200D816B90320BDE8F8832068C06850
:1034F00000F00400F8B1802D1ED0402D1CD02068B3
:103500000068C0F3C000B0B100BF00200090206888
:103510000068009020684068009000BF00BF20460F
:10352000FFF7C6FD0820606400BF002084F840005B
:1035300000BF0120D8E7FFE7206800682840A842C4
:1035400001D1012000E00020B842C3D00020CBE729
:103550000021044A1268D1B241EA0022014B1A60EC
:10356000704700000C18014010B50248FEF790FCAF
:1035700010BD00001801002010B50248FEF788FCBD
:1035800010BD0000FC0F002000BFFEE700B585B0B5
:1035900000BF00BF0C48806940F004000A49886100
:1035A0000846806900F00400009000BF00BF00BF23
:1035B00001200190029003900320049001A9034888
:1035C000FDF79EFD05B000BD00100240000801405F
:1035D00010B5044600BF00224FF480411648FDF7A5
:1035E00041FF00BF00BF012211031348FDF73AFF5E
:1035F00000BF2046FFF7ACFF00BF00224FF4006180
:103600000D48FDF72FFF00BF00BF00224FF400510F
:103610000948FDF727FF00BF00BF012251030648FC
:10362000FDF720FF00BF00BF0122D1020248FDF7D5
:1036300019FF00BF10BD0000000C014010B504468A
:1036400000BF012291031648FDF70CFF00BF00BF29
:10365000012211031248FDF705FF00BF2046FFF7C6
:1036600077FF00BF00224FF400610D48FDF7FAFE1E
:1036700000BF00BF00224FF400510948FDF7F2FEE1
:1036800000BF00BF012251030548FDF7EBFE00BF5C
:1036900000BF0122D1020248FDF7E4FE00BF10BDC9
:1036A000000C014002480068C0F30220704700008F
:1036B0000CED00E010B5002804DB0A07130E054AE4
:1036C000135406E00A07140E034A00F00F031B1FF1
:1036D000D45410BD00E400E018ED00E000BF7047D6
:1036E00008B1072900DB704700F10C0343F82120E3
:1036F00000BFF8E770B504467CB10848006860B1C7
:103700002579092D08D205EB4501054A02EB810117
:10371000087A02490968884700BF70BD240000206C
:103720008C3D000870B5044600BF2079A168884729
:103730000546E07800F00700002802DD2088401CE4
:103740002080E078B5EBD01F13D0E078C008401C93
:10375000E17860F3C501E170C1F3C20003280CDB1E
:10376000E07865F3C710E070E07820F03800E07092
:1037700003E0E07820F03800E070E07800F0070027
:1037800005287DD2DFE800F0032858AFDB00E078A1
:10379000C0F38010E178B0EBD11F17D1A07820F0F2
:1037A000F000A07000BFE06810B12046E1688847D3
:1037B00000BF00202080A07820F00F00401CA070E7
:1037C000E07820F00700401CE07004E0A07820F0D2
:1037D000F0008030A070DBE0E078C0F38010E1788A
:1037E000B0EBD11F13D0A07820F0F0001030A07003
:1037F00000BF206910B120462169884700BF002022
:103800002080E07820F00700801CE07013E0208822
:10381000C82810DDA07820F0F0005030A07000BF64
:10382000206A10B12046216A884700BFE07820F066
:103830000700001DE070ABE0E078C0F38010E17895
:10384000B0EBD11F25D1A07820F0F000A07000BF10
:10385000E06810B12046E168884700BFA07800F01A
:103860000F000F2804DAA078411C61F30300A07058
:1038700000BF606910B120466169884700BF00E061
:1038800081E000202080E07820F00700C01CE0707C
:1038900028E020883C2825DDA07800F00F000128D2
:1038A0000BD1A07820F0F0003030A07000BFA069EC
:1038B00010B12046A169884710E0A07800F00F0001
:1038C00002280BD1A07820F0F0004030A07000BF9B
:1038D000E06910B12046E169884700BFE07820F038
:1038E0000700E07054E0E078C0F38010E178B0EBBE
:1038F000D11F1BD0A07820F0F0001030A07000BFC6
:10390000206910B120462169884700BF20883C28E3
:1039100007DA00202080E07820F00700801CE070AB
:103920000CE0E07820F00700E07007E020883C28F9
:1039300004DDE07820F00700401CE07028E0E0782B
:10394000C0F38010E178B0EBD11F0BD1A07820F04C
:10395000F0006030A07000BF606A10B12046616A5C
:1039600088470FE0A07820F0F0001030A07000BF72
:10397000206910B120462169884700BFE07820F017
:103980000700E07004E0E07820F00700E07000BF7E
:1039900000BF70BD2DE9F04104460D4616461F4696
:1039A00004B10DB9BDE8F0812C212046FCF7B9FC2B
:1039B000A07820F0F0008030A070A5600EB9012042
:1039C00000E00020E17860F3C711E170E07866F371
:1039D0008610E0702771E07820F00700E07000BFEB
:1039E000E0E7000070B5044604EB4402064B33F8F0
:1039F000221004EB440203EB82025068FDF720FD25
:103A00000546284670BD00008C3D0008014611B9EE
:103A10006FF0010070470948026805E08A4202D150
:103A20004FF0FF30F6E7926A002AF7D103480068AA
:103A30008862024801600020ECE7000030000020AE
:103A400010B50548046803E02046FFF76BFEA46A42
:103A5000002CF9D110BD00003000002001490860A1
:103A6000704700000C00002010B504464FF47A7136
:103A700004FB01F000F002F810BD000070B5034631
:103A800000224FF0E02675690D4E366803FB06F400
:103A90004FF0E026B16910E04FF0E026B0698842AF
:103AA0000BD0884202D20E1A324402E02E1A0E4483
:103AB00032440146A24200D300E0EDE700BF70BDF2
:103AC0000C00002038B504460D4600BF00BF124868
:103AD000C06940F001001049C8610846C06900F0A3
:103AE0000100009000BF00BF00BF88040B490860C0
:103AF0000846456000218160C460FEF7FBF80022A3
:103B000002211C20FDF711FD1C20FDF7FEFC0348DF
:103B1000FEF724F938BD0000001002409401002097
:103B2000FDF7B8FC4FF4E01000F048F84820FFF72C
:103B300095FFFEF7FDFDFEF709FDFFF727FDFEF7F8
:103B40003BFF41F61F413120FFF7BCFF1548FEF750
:103B50005BFDFEF7E7FEFEF70FFF22E0124800785C
:103B6000012809D111480078012805D100200F490A
:103B700008700120FEF7AAFE0B4801780C48007877
:103B8000FEF7D6FF08490870002009490870094867
:103B900000680949884204D9FDF71AFD002005494B
:103BA0000860DBE7F525000806000020040000207F
:103BB000050000200000002040420F0030B58FB00B
:103BC00005460124282105A8FCF7ABFB1421684613
:103BD000FCF7A7FB01200590000406900020079049
:103BE00002200C90C1030D910E9505A8FDF736FE3D
:103BF00004460CB100BFFEE70F20009002200190A8
:103C0000002002904FF48060039000200490022175
:103C10006846FDF7FFFC04460CB100BFFEE70FB09D
:103C200030BD000000000000000001020304060790
:103C3000080900000000010203040203040506074E
:103C400008090A0B0C0D0E0F1010010200140140A0
:103C500040000001030000000100000000140140CA
:103C600020000001030000000100000000140140DA
:103C700010000001030000000100000000140140DA
:103C800008000001030000000100000000140140D2
:103C900004000001030000000100000000140140C6
:103CA00002000001030000000100000000140140B8
:103CB00001000001030000000100000000100140AD
:103CC0000010000103000000010000000008014096
:103CD0000010000103000000010000000008014086
:103CE000000800010300000001000000000801407E
:103CF0000004000103000000010000000008014072
:103D00000002000103000000010000000008014063
:103D1000000100010300000001000000001001404C
:103D2000000200010300000001000000001001403B
:103D3000000100010300000001000000001001402C
:103D40008000000103000000010000000018014095
:103D500008000001030000000100000000180140FD
:103D600010000001030000000100000000180140E5
:103D700004000001030000000100000000180140E1
:103D80002000000103000000010000000F000000FF
:103D9000000C0140010000000B0000000014014075
:103DA000020000000A0000000014014003000000AF
:103DB0000D00000000140140070000000800000092
:103DC00000140140080000000C0000000014014035
:103DD000040000000E000000001401400500000077
:103DE0000900000000140140060000000F00000060
:103DF000001401400900000000C1814001C0804161
:103E000001C0804100C1814001C0804100C18140AA
:103E100000C1814001C0804101C0804100C181409A
:103E200000C1814001C0804100C1814001C080418A
:103E300001C0804100C1814001C0804100C181407A
:103E400000C1814001C0804100C1814001C080416A
:103E500001C0804100C1814000C1814001C080415A
:103E600001C0804100C1814001C0804100C181404A
:103E700000C1814001C0804101C0804100C181403A
:103E800000C1814001C0804100C1814001C080412A
:103E900001C0804100C1814000C1814001C080411A
:103EA00001C0804100C1814001C0804100C181400A
:103EB00000C1814001C0804100C1814001C08041FA
:103EC00001C0804100C1814001C0804100C18140EA
:103ED00000C1814001C0804101C0804100C18140DA
:103EE00000C1814001C0804100C1814001C08041CA
:103EF00001C0804100C1814000C0C101C30302C2B2
:103F0000C60607C705C5C404CC0C0DCD0FCFCE0E19
:103F10000ACACB0BC90908C8D81819D91BDBDA1A89
:103F20001EDEDF1FDD1D1CDC14D4D515D71716D6F9
:103F3000D21213D311D1D010F03031F133F3F23269
:103F400036F6F737F53534F43CFCFD3DFF3F3EFED9
:103F5000FA3A3BFB39F9F83828E8E929EB2B2AEA49
:103F6000EE2E2FEF2DEDEC2CE42425E527E7E626B9
:103F700022E2E323E12120E0A06061A163A3A26229
:103F800066A6A767A56564A46CACAD6DAF6F6EAE99
:103F9000AA6A6BAB69A9A86878B8B979BB7B7ABA09
:103FA000BE7E7FBF7DBDBC7CB47475B577B7B67679
:103FB00072B2B373B17170B05090915193535292E9
:103FC00096565797559594549C5C5D9D5F9F9E5E59
:103FD0005A9A9B5B99595898884849894B8B8A4AC9
:103FE0004E8E8F4F8D4D4C8C448485458747468639
:103FF0008242438341818040184000080000002035
:10400000500000006C0100086840000850000020CB
:10401000E82F0000880100080000000000000000F8
:104020000024F40000000000000000000000000078
:10403000000000001000000001000000000000006F
:104040000000000000000000000000000000000070
:104050000000000000000000000000000000000060
:08406000000000000000000058
:0400000508000131BD
:00000001FF
